:020000040000FA
:0200000078285E
:06000A0082070C340E34E5
:1000100011341034103411340E3480340C340E3456
:1000200010340E34013411340E3480340C341F3447
:1000300002340434083410341F34803480340C34D7
:100040000E341034103411340E34803480340C34B7
:100050000E3410340E3401340E34803480340C34B9
:100060001F340234043408341F34803400341B3409
:100070000E3404348234043408341F3480340034A1
:1000800062347934203453342034353420343534D8
:100090002034573420345434003444347534053417
:1000A00069346C346E346934203404346C3465340F
:1000B0006E34003444347534053465346E346A3437
:1000C000653420340034523461347A346C34693409
:1000D0006B346134203400348207303431343234AC
:1000E00033343434353436343734383439342034D6
:1000F00003018501860189010D219A00890A0D21DC
:100100009C00890A0D219200890A0D219B0083160B
:100110004230810085010F308600831286214830ED
:1001200073210301AD210C30732101307321FA30AA
:10013000A5214730AD21C03073213A30AD21552182
:1001400001307321FA30A5213021A720C62080304C
:1001500073215430AD21893073211A084521C030F4
:1001600073215D30AD212D30121C2030B721C930F4
:1001700073211B084521080006190800061DBE282A
:100180001A089C009B01EF20A7200800BC2006084D
:100190000339033C031DC628BC2006080339033C71
:1001A0000319CC280618D628E720D728EB20BC2036
:1001B00006080339031DD728BC2006080339031994
:1001C000DC280618E528EB20C628E720C6281221DF
:1001D000EF20A72008002121EF20A7200800890197
:1001E0001A0888000121890A1C0888000121890A4F
:1001F000120888000121890A1B088800012130218A
:1002000008008316081555308900AA308900881423
:10021000881808290811831208008316081483120D
:10022000080808003F301A02031908009A0A121041
:100230001C081A029B000318080012149B099B0A51
:10024000080001301A02031C080012109A031C084F
:100250001A029B000318080012149B099B0A08004D
:100260001A089D003F301D0203189D168316860153
:1002700083121D0886000514000000000510860189
:1002800083160F30860083120800622114080319B8
:100290000A306C20B72115086C20B7212030B72117
:1002A0006430B7214230B721080010309700473042
:1002B0009800FD309900990B5B29980B5B29970BEF
:1002C0005B29080095009301940164301502031C1A
:1002D0006C299500930A65290A301502031C080051
:1002E0009500940A6C298C00F03086040C080F38B5
:1002F00086058121F03086040C0E0F388605812199
:100300000800051505110130A52108009630A5212A
:100310003030860081212930A52181218121293099
:10032000A521203086008121812180308600812115
:100330000130A5218601812180308600812186013E
:100340008121F03086008121080090001D308F004F
:100350008F0BA829900BA6290800910011080520F1
:10036000003E03190800B721910FAE2908008C0048
:10037000F03086040C080F38860585158121F03091
:1003800086040C0E0F388605860081218511080031
:02400E00F13F80
:084200000000000000000000B6
:00000001FF
